:100000008A110A120528000009000730990083169A
:10001000051085100511051285128312F430A00019
:100020000130A10013220514F430A0000130A1001A
:10003000132250210510F430A0000130A10013223A
:100040000516F430A0000130A10013225021051242
:10005000F430A0000130A10013228516F430A00076
:100060000130A100132258202C30A0000130A10043
:10007000132201228512AC012C08053C031C5428D4
:10008000AD012D083B3C031C4E28E830A000033096
:10009000A10013220130AD07031C41281F30830546
:1000A0000130AC07031C3C281F3083050E2857285D
:1000B0000721932093209C2093209320AC012C08AF
:1000C000023C031C7B28B620D120102119210721D6
:1000D000A420C820BF20AD012D08023C031C7528B8
:1000E0008A200130AD07031C6C281F3083050130C6
:1000F000AC07031C5F281F308305DA20E3201021A2
:1001000022212B210721EC20F520AD2093209320E4
:1001100093200800422142214221342142214221E0
:10012000342134210800422142214221422134213C
:100130004221342134210800C820FE20C820FE209E
:10014000C820FE20C8200800422142213421342149
:100150003421422134213421080042213421342128
:10016000342134214221342134210800422142210A
:1001700034214221422134213421342108004221FA
:1001800042214221342134213421342134210800F8
:10019000422142213421422134214221342134217F
:1001A00008004221342134213421422142213421CA
:1001B00034210800422142213421422134213421BA
:1001C00034213421080042213421422134213421B8
:1001D000422134213421080042214221422142217E
:1001E0004221342134213421080042213421342198
:1001F000422134214221342134210800422134217A
:100200004221342142213421342134210800422169
:100210003421342134213421342134213421080083
:10022000422134213421422134213421342134210A
:100230000800422134213421422142213421342139
:100240003421080042214221342134214221342129
:1002500034213421080042214221422142214221FD
:100260003421342134210800053084000230AA00F2
:100270005730A0000130A1002030A2000030A300C0
:100280004E220800053084000230AA008730A0000A
:100290000130A1001C30A2000030A3004E22080053
:1002A0009121BB219121BB219121C921A821A82104
:1002B000A8218021BB218921BB219621BB21A2211C
:1002C000BB217E21BB2184216D21C921012208008F
:1002D000F021DF21F021DF210800F021DF21F021D2
:1002E0000800DF21F021DF21DF210800DF21F021DC
:1002F000DF210800DF21DF21F0210800F0210800C4
:10030000F021F021DF210800DF21F021F021F02190
:100310000800DF21DF21F021DF210800F021F0219A
:100320000800DF21DF21DF21F0210800F021F0218A
:10033000F021F021F0210800DF21DF21F021F02160
:10034000F0210800DF21DF21DF21DF21DF2108008C
:100350007121BB217A21BB219C21BB216821BB21BA
:100360007621BB218E21C921080005113C30A00057
:10037000A1011322080005113C30A000A1011322A5
:100380003C30A000A10113223C30A000A1011322A7
:10039000080005113C30A000A10113223C30A00050
:1003A000A10113223C30A000A10113223C30A00087
:1003B000A10113223C30A000A10113220800051561
:1003C000053084000230AA00F330A0000130A10003
:1003D0003C30A2000030A3004E220511B5210800D8
:1003E0000515053084000230AA00F330A00001306A
:1003F000A100F030A2000030A3004E220511B5216B
:1004000008000515053084000230AA00F330A00072
:100410000130A100DC30A2000530A3004E220511FE
:10042000B5210800122AA00803191E2A2522A003BC
:1004300000000000000000000000132AA1080319BA
:1004400008002522A103A003132A0C30A500A50B48
:10045000272A000000001230A200A20B342A362204
:10046000362200000000080036222D2A0D30A4009C
:10047000A40B382A000008001030A8020001031C59
:10048000013EA902031C0800452A0A30A802000107
:10049000031C013EA902031C0800452A2A08800407
:1004A0002008A8002108A9003C220130A202031C58
:1004B000A3032A0980052008A8002108A9003C22DE
:0E04C000A208031D4E2AA308031D4E2A0800A1
:02400E00A4010B
:00000001FF
